:030000000219FDE5
:03000B000200A848
:03002B000201547B
:03005B000202DEC0
:030073000202C4C2
:1000800002030406080C10182030406080040608A3
:100090000C10182030406080A0C000070F1F3F05E3
:1000A000050D050305030302C2AFC0D0C0E0206206
:1000B00017E5256002E473E525F4F58A758B00D217
:1000C00062D0E0D0D0D2AF3285268AC262E526F473
:1000D0006035306803207210758B00D0E0D0D0D22C
:1000E00095D293D297D2AF32D295D293D297206E37
:1000F0000C206609740CD5E0FDE57E4290758B00FE
:10010000D0E0D0D0D2AF32758A00C28DD26201FD6C
:1001100001B7306805206602C29501B73068052036
:100120006602C29701B7306805206602C29301B724
:10013000C294306805206602C29501B7C296306845
:1001400005206602C29701B7C29230680520660298
:10015000C29301B7C2AFC2AD53E6EFC0D0C0E0D288
:10016000D3D2AFC2CEE52A6007207449152A21B543
:100170007800790020742EE580307E01F430E502AD
:1001800078FF53DACF207E0343DA20307E0343DA50
:1001900010C2D8C271E580307E01F430E50279FFEB
:1001A000C3E89970CB306103752A18207403752A4F
:1001B00018885FD27020740DE52B6004152B21C5C3
:1001C00043DA01C2D82070024127A85F206102C231
:1001D00070207431C3E894F0400374F0F8E8C4541C
:1001E0000F28F87984B703024105C313C31387218D
:1001F000200802C313200A06C3C898F8410528F84E
:10020000500374FFF8C3E895685003E568F8882246
:10021000E52D54066011E533C313C31324062522CC
:10022000F52250037522FF852224A824C3E52495D6
:10023000644002A8648825E5697002416BC3E8AA9E
:10024000699A5003E8FAE4F9EAC333FBE56BF45B1F
:1002500029400D256AF8E56A6002156A400B416B7A
:100260000AC3E56A9A5002056A78FF8826C26EC3FF
:10027000E52694F84002D26EC3E52594404002D2B0
:100280006420CF0AD0E0D0D043E610D2AD32C2CF46
:10029000053A7801E52A6005307402152AC3E55F46
:1002A0009401400575620041BA756300756C00E504
:1002B000622401F56250037562FFD0E0D0D043E6BE
:1002C00010D2AD32C2AFC0D053E67FC2607591008C
:1002D000855694855795759104D0D0D2AF32C2AF70
:1002E00053E6EFC2ADC0D0C0E0C0F0D2D3D2AFA8C9
:1002F000FBA9FCC2D8307102614553DACF207E03DE
:1003000043DA10307E0343DA20D271E580307E017B
:10031000F420E502611C88278928A17253DACF20D6
:100320007E0343DA20307E0343DA10C2D8C2713034
:100330007402A15E7800E580307E01F430E502A110
:100340005E885FA14653DACF207E0343DA20307EF9
:100350000343DA10C271206102811E53DACF207E7E
:100360000343DA10307E0343DA20C2D8D271885AB0
:10037000895BC3E89558F8E99559F97B007E087ABE
:1003800000C3E8948CE994005005755E00811088E4
:100390002178A2E6A8216055C3E894C8E9940050EA
:1003A00008E4D2E4FB7A0A61EBC3E89468E99401BB
:1003B0005008E4D2E3FB7A0F61EBC3E894D0E994F0
:1003C000025008E4D2E2FB7A1E61EBC3E894A0E994
:1003D00094055008E4D2E1FB7A3C61EBC3E89498C1
:1003E000E994085008E4D2E0FB7A787E00C3E895EF
:1003F0005CFCE9955DFD30E70AECF42401FCEDF4CA
:100400003400FD755E00C3EC9AED9E5003755E01ED
:10041000885C895D855A58855B597802A146C3E896
:100420009527F8E99528F9307C02A12A307B02A1B2
:100430002A307A02A1232075028141E9FDE8FC817E
:1004400060E9C313F9E813F8307902A123E9C31373
:10045000F9E813F8307802A123E9C313FDE813FC8F
:1004600020612CC3EC941CED940240028177ED7066
:0F0470001EC3EC94C850180529E5297002152900
:10047F00C3E529940A5002A15E755F00D270A15E98
:10048F00E529600215297888E6F97400207F08783D
:10049F0096B90302789EE624FAFEE43400FFC3EC1B
:1004AF009EFCED9FFD9208B90310A208500720761D
:1004BF0009D27681C9307602C276A2085016B903E6
:1004CF000DECF42401FCEDF43400FD0204E378009C
:1004DF007900A12AB90315EC33FCED33FDC3EC947D
:1004EF000AFCED9400FD50047C007D00C3EC94FFEA
:1004FF00ED9400400678FF7900A12AEC8575F0A4F1
:10050F00C5F0A2F733F87900400302054678FF796A
:10051F0000020546E9C313F9E813F8307C0EE960D1
:10052F000278FFC3E81338F8E43400F9C3E894FF06
:10053F00E99400400278FF885FD270206102A15ECB
:10054F00741FF4552F4BF52FC274EB7002D27475D4
:10055F002A18307403752A0A306102A172207403BD
:10056F0053DAFE207403752B06D0F0D0E0D0D0D232
:10057F00AD43E6103279010205A279030205A27993
:10058F000A0205A2791E0205A279640205A279C8A2
:10059F000205A27817E4D5E0FDD8FAD9F6227A142D
:1005AF007B780205C97A107B8C0205C97A0D7BB462
:1005BF000205C97A0B7BC80205C97902B27DE4C274
:1005CF0096D5E0FDC297D5E0FDD297D5E0FDD29646
:1005DF00D5E0FDC295E576D5E0FDD2957496D5E0D0
:1005EF00FDD9D9EAF8D5E0FDD8FBDBCEC29622C300
:1005FF007C007D0075F00005F0EA33FAEB33FB5019
:10060F00F6EB13FBEA13FAC3E9FFE8FEE89AF8E901
:10061F009BF95004EFF9EEF8B3EC33FCED33FDD555
:10062F00F0DFEDF9ECF822E889F08A20D2D4F8A9AE
:10063F00F07B0030F70B7BFFF42401F8E9F4340072
:10064F00F9E88520F0A4ADF0F8E98520F0A4AFF02B
:10065F00FEED2EF974003FFA7C04C3EA13FAE91396
:10066F00F9E813F8DCF48BF030F70AE8F42401F81A
:10067F00E9F43400F9E889F0C2D4F8A9F02222C3D2
:10068F00E54113F9E54013F8C3E54598F8E54699B8
:10069F00F9500CC3E89480E994FF40160206C5C3D5
:1006AF00E8947FE9940050030206C5787F79000231
:1006BF0006C5788079FF884A894B22E54A2547F895
:1006CF00E54B3548F9854B20E4300701F43549FAFD
:1006DF0030E709C3EA94F04015020703C3EA940F09
:1006EF00500302070378FF79FF7A0F0207037800A0
:1006FF0079007AF0C3E5249564500AC374019524F8
:10070F00500B020721E54B20E70E020721E54B3086
:10071F00E706884789488A492278A4E6FAC3E54A5A
:10072F0033F8E54B33F9D136E930E70BC3E8948062
:10073F00E994FF4013E15BC3E8947FE99400500212
:10074F00E15B787F7900E15B788079FFE820E7153E
:10075F00C3E52398F84009C3E894014003020782D8
:10076F007801020782E8F424012523F840030207E9
:10077F008278FF884C2278A5E6FAA848A949D13695
:10078F00E930E70CC3E89401E994FF40160207B67D
:10079F00C3E894FFE9940050030207B678FF79008D
:1007AF000207B6780179FFE920E715C3E54C98F801
:1007BF004009C3E8940140030207DD78010207DD19
:1007CF00E8F42401254CF840030207DD78FF882464
:1007DF002278FFC26420693D206A12D264C3E541CA
:1007EF00940A4009C3E52594405002C26479A1E7F9
:1007FF006023E541601F74FF8541F0848539F03037
:10080F006A0375F005A4F8C5F0600278FFC3E89598
:10081F00675002A867886622C3E5409440E541947B
:10082F0001E5665003140138046002F566220208E0
:10083F00402275E890227883E6FFE5E820ECF7A8E0
:10084F00BDA9BE0573C3E57394084052757300E9E3
:10085F00FA79A0E76044EA7007E574601B02087B31
:0D086F00C3E895746010E5745006600C1429
:10087C000208870460F9020887E574F574C3946D67
:10088C00401B7564C0C394044013756480C3940406
:10089C00400B756440C39404400375640075BB0839
:1008AC0022E564F460020564E573B4070375BB10BC
:1008BC0022743279A687F0A4C5F0A2F733F8C3E806
:1008CC0095644002A8648822882488258826886735
:1008DC00227540007541F022C2AF75C820A8CCA982
:1008EC00CDAA3A30CF010A75C824D2AFAB3BAC3C91
:1008FC00883B893CC3E89BF8E99C206908F9306780
:10090C000221F92156AD3D8A3DF9EA9DFA60047841
:10091C00FF79FFAE3EAF3F8B3E8C3FC3EC9FFCC3D9
:10092C00E99CF542A83BA93CC3E89EF8E99FF9C3B2
:10093C00E54113FBE54013FAE82AF540E93BF541A4
:10094C0050067540FF7541FF21A0AA40AB41AC4059
:10095C00AD417E047F02C3EB940440021E1FC3EB27
:10096C00940840021E1FC3ED13FDEC13FCDEF7C30D
:10097C00EA9CFAEB9DFBEF6009C3E913F9E813F865
:10098C00DFF7EA28FAEB39FB8A408B4150067BFFF4
:10099C008B408B41C3EB94025002D2673069047FC9
:1009AC000321CB7892E6FFC3E537948240110FC345
:1009BC00E53794A040010FC3EF940640027F057EFB
:1009CC0005E541C4540FF9E541C454F0F8E540C4C1
:1009DC00540F28F8C3E89EFAE99400FB4009C3EAD7
:1009EC009402EB940050047A02E4FB4145AA40AB1C
:1009FC0041EBC4FEEAC4540F4EFCC3EA9CFAEB94E0
:100A0C0000FBC3E813C313F8EA28FAEB3400FB8AA3
:100A1C00408B41C3EB94024002C2677805EBC4FEE5
:100A2C007B00EAC4540F4EFAC3EA98FA4005C3940B
:100A3C000250027A027892E6FF30600241458552FC
:100A4C0056855357D26043E680C3E49AF8E49BF989
:100A5C0030670241DFE8FAE9FBD3E913FDE813FC48
:100A6C0088528953C3EF94036038EF20E00DE82CD3
:100A7C00F8E93DF9ECFAEDFB020A9AE828F8E939B5
:100A8C00F9C3E82402F8E93400F97AFE7BFFC3EFDE
:100A9C009403400E8A548B55884E894F8C508D513F
:100AAC006113885489558A4E8B4F8C508D51306907
:100ABC0020C3E53394034019E542A2E713F8E5554A
:100ACC00F4240138400B20E7087554FFF42401F599
:100ADC00556113E8FAD3E813FC8852C3EF94036012
:100AEC0020EF20E007E82CF8ECFA41FFE82824027C
:100AFC00F87AFEC3EF940340088A54884E8C5061F8
:100B0C001388548A4E8C50E56BC3335002646BF5DA
:100B1C006B306002611D753402D26043E680E52DB6
:100B2C0054066026A840A941C3E913F9E813F8C29A
:100B3C00AF53E67F759100C3E498F594E499F5956D
:100B4C00759104D26043E680D2AF22D26575440021
:100B5C00752000306B03752040020B76D26575440E
:100B6C0000752040306B03752000D2AF78012067F0
:100B7C0022E52D54066002C265C3E541940540137D
:100B8C007802940540087803940540027806306991
:100B9C0002780A206019E544601530690AC3E53310
:100BAC0094034003D53406D2AFD26C81477125D261
:100BBC00AF0000C2AF206726E541C3FB940F400293
:100BCC007B0FEB240530730123306A0274282062FA
:100BDC000123F93069027982E58BC39940B505444C
:100BEC00E59B5440B52002813130690A08C3E89472
:100BFC000A400108619F2065026176C26553E67F59
:100C0C007591003067107594007595FE759104D23E
:100C1C006043E6806176AE40AF41C3E49EF594E458
:100C2C009FF5958118C3E5339402500261763065C7
:100C3C00026176D8028145619FC26C53E67F759143
:100C4C0000855494855595759104854E56854F575E
:100C5C00D26043E680D2AFE52D54066008206A02CC
:0E0C6C000533020C81306C0D206B0A206507E9
:100C7A00158115810214FE22780030640530650260
:100C8A007801E53775F007A4F9E5F028F5F0E9A24F
:100C9A00F013A2F113A2F213F537C3947850037537
:100CAA003778C3E53795384008D266D295D293D2C1
:100CBA009730600281BB855056855157D26043E612
:100CCA008022207D11C2AF754302C296D294D2AF60
:100CDA00759F11020E9BC2AF754302C296D292D281
:100CEA00AF759F11020E9B307243207D20C2AF75F3
:100CFA00430390013C757E40D293C292306204C293
:100D0A0097A10FD296D2AF759F13020E9BC2AF75F1
:100D1A00430390013C757E40D295C294306204C26E
:100D2A0097A12FD296D2AF759F10020E9B207D17E6
:100D3A00C2AF75430390011CD293306202C297D2AC
:100D4A00AF759F13020E9BC2AF75430390011CD26D
:100D5A0095306202C297D2AF759F10020E9B207D1A
:100D6A0011C2AF754304C294D292D2AF759F1002DA
:100D7A000E9BC2AF754304C292D294D2AF759F1331
:100D8A00020E9B307243207D20C2AF75430590014D
:100D9A0030757E10D297C296306204C295A1ABD24A
:100DAA0094D2AF759F11020E9BC2AF754305900195
:100DBA0048757E04D297C296306204C293A1CBD200
:100DCA0092D2AF759F11020E9B207D17C2AF754359
:100DDA0005900112D297306202C295D2AF759F1167
:100DEA00020E9BC2AF754305900126D2973062EB83
:100DFA00C293D2AF759F11020E9B207D11C2AF75AF
:100E0A004306C292D296D2AF759F13020E9BC2AF0F
:100E1A00754306C294D296D2AF759F10020E9B30CC
:100E2A007242207D20C2AF754301900148757E044D
:100E3A00D295C294306204C293C147D292D2AF759E
:100E4A009F10020E9BC2AF754301900130757E1050
:100E5A00D293C292306204C295C167D294D2AF755E
:100E6A009F13C19B207D16C2AF754301900126D204
:100E7A0095306202C293D2AF759F10C19BC2AF7503
:100E8A004301900112D293306202C295D2AF759F8C
:100E9A0013C26622900110757E00D295D293D29722
:100EAA00C294C292C296C26222788076FF0876FF06
:100EBA000876FF0876FF08760308760408760A089B
:100ECA007603087601087601788C76010876FF08A1
:100EDA0076FF0876FF0876FF0876FF08760308761D
:100EEA00FF0876FF0876FF0876250876D00876FA96
:100EFA000876FA0876040876FF087601087600086C
:100F0A00767A0876FF087601087601087600087670
:100F1A0003227887E6FFC272BF0302D2727888E69C
:100F2A00C394036008C27DE630E102D27DC27E78B6
:100F3A0089E630E102D27EC3EF94026008758E0121
:100F4A00D273020F54758E00C273227880E6149011
:100F5A0000809378A4F67881E6149000809378A5AF
:100F6A00F67886E61490008D9378A6F6789CE67556
:100F7A0038FF75390CB402067538A075390AB403FE
:100F8A000675388275390578A3E61490009A93F5A8
:100F9A0069D19E22227896E6FA7897E6FB7888E667
:100FAA00B40305C3EB940EFB307F047A007BFFC3C6
:100FBA00EB9AFCC3948250027C827575000575EC2D
:100FCA008575F0A4C3E5F0947D40F222D27FF19FAB
:100FDA001205937A007B007C10120589E55F2AFAD4
:100FEA0074003BFBDCF37C04C3EB13FBEA13FADC6F
:100FFA00F7FEC27F120F9F22E5EF20E6037520005D
:10100A000520903FFFE520146006901DFF14600044
:10101A009304600375EF1253D9BF7581C043FF80F3
:10102A0012058475EF0243B203E5B3240420E70DE9
:10103A00F521E5E320E0068521B343E301120E9E84
:10104A007580FF75A40075F1B275D4DF7590A97526
:10105A00A5FC75F2FE75D50175A60175E241E4F8A5
:0E106A00F6D8FD756B01120EB3121540789882
:101078008676753001C2AF12059D1205AD12059333
:101088001205B41205931205BB12059312165912D4
:10109800059D12059D120598C2AF78FA79FA308538
:1010A80007D9FBD8F7021C00120F1C120F55120F9C
:1010B8009E120F9F78988676120E9E7588507589B5
:1010C8001275C82475910475D84075A82275B802A0
:1010D80075E690759B80759D0075D10E75BC587529
:1010E800BB0875BA1175E880120584D2AF12083DA5
:1010F80053DACF207E0343DA20307E0343DA1043ED
:10110800DA01C2D8C27112059DD2617B037A0CE55F
:101118005E70077A0CDB030210A01205932070039F
:101128000210A0C270E55FC3940240E1E52F541F8E
:10113800856160F561B560D5DAD5C26153DACF2033
:101148007E0343DA20307E0343DA10C2D8C27178B6
:10115800A2E67008D274E52F54E0F52FC275752900
:1011680000120598307409C3E529940A4002D27523
:1011780012058978023074027800C3E55F9840F060
:10118800C2AF1205AD1205AD1205ADD2AF12059D65
:10119800754D007888E6B403024180120589788C81
:1011A800E6C394015003021280E530C39401500352
:1011B800021280207435C3E55F94FF500302128049
:1011C800C2AF1205C2D2AF120598C3E55F940150B1
:1011D800EFC2AF1205AD12058E1205ADD2AF1205E2
:1011E80098C3E55F94FF40E90216DE7F05D27F12BF
:1011F8000F9F120598C2AFC27F120F9FAE5FC3E563
:101208005F947FD2AF407B120584C2AF1205C2D271
:10121800AFDFDA120FD6C3EE94057897F612059D64
:101228001215821216617F0AD27F120F9F1205983B
:10123800C2AFC27F120F9FAE5FC3E55F947FD2AF8C
:1012480050E4120584C2AF1205AD12058E1205AD29
:10125800D2AFDFD4120FD6EE24057896F612059D8C
:10126800121582121690120598120F9FC3E55F940B
:10127800FF500221BB0216DEC3E55F954D40038592
:101288005F4D12059878017988E7B403027805C3A1
:10129800E55F984002219BC2AF1205C21205C21237
:1012A80005C2D2AF12059D753000E4F531F532055F
:1012B80031E531F470390532789AE67819146012FC
:1012C800783214600D787D14600878FA146003751C
:1012D8003200C3E53298401715327531B4789986D3
:1012E80076C2AF1205C2D2AF7898867612059812E8
:1012F800058EE52A700530740201A0780120740279
:101308007806C3E55F9840A77888E6C3940360032E
:10131800120598E52A70030210A0C2AF120E9EE4CF
:10132800F522F523F524F525F526F56AD2AF78855B
:10133800E6C333F568E4F545F546F547F548F5495C
:10134800F573F52CF52DF53775730875BB10120577
:1013580084120841E5E820ECFBA8BDA9BEE97001AC
:10136800F8887412084575730875BB107887E6FE0F
:101378007602120F1C7887EEF6C2AF7564FF12086A
:10138800BD852264852265852266D2AF75220175E6
:10139800240175250175260185636C756D017888B2
:1013A800E6B40307C27D307602D27DD268D2697571
:1013B8003300120E04120E291208DD1208E4120876
:1013C800DD1208E41208DD0213DFC2AF120F1CD2CF
:1013D800AF75730075BB08120B6812068D120C826C
:1013E800120CCC1208E4120B57306D0312068E2033
:1013F80067031207E0306703120827120C82120CE9
:10140800F11208E4120B68306D031206CA120C823E
:10141800120D681208E4120B57306D0312072812D8
:101428000C82120D8D1208E4120B68306D0312073E
:1014380085120C82120E041208E4120841120B578E
:10144800120C82120E291208451208E43069322063
:101458006B2F85676485676585636C756D01791881
:0E1468007A0CC3E53399400CC269D26A8A350A
:101476007564FF021489C3E55F940140030213DF1C
:10148600021506306A1B206B18E535147004C26A13
:1014960061D2F535C3E55F940140030213DF0215FF
:1014A60006753600C3E5627882985054307404E5B8
:1014B6002A604D7888E6B40317207D0520760781DB
:1014C600D630760281D6206B07D26B856764811E83
:1014D60078F0306B058567647820C3E54198500243
:1014E60061DF306B1BC26BC27D307602D27DD26A61
:1014F60075351285676461DF0536E55F6002A1090F
:10150600753600C2AF120E9E7887E6FE7602120F7F
:101516001C7887EEF6E4F522F523F524F525F52665
:10152600F568C268D2AF120584120E9E307409C3E4
:10153600E5369405400201A041B2901A0D782012BA
:1015460015C4E520B45A0CA31215C4E520B4A503AE
:10155600021562120EB3121582021581901A0378D3
:10156600807B0A1215C4A308DBF9901A0F788C7BCE
:10157600181215C4A308DBF9901A2722C2AF121657
:10158600031215DD901A00740E1215C9A374041205
:1015960015C9A374141215C9901A0378807B0A1210
:1015A60015C8A308DBF9901A0F788C7B181215C89A
:1015B600A308DBF91216161215F4901A2722E493E3
:1015C600F622E6438F01538FFD75EF0275B7A575B9
:1015D600B7F1F0538FFE22438F02438F0175EF025E
:1015E60075B7A575B7F1901A0DF0538FFC22901AB6
:1015F6000D745AB1C9901A0E74A5B1C9227A307900
:10160600D07820901A40B1C4E520F709A3DAF72272
:101616007A3079D0901A40E7B1C909A3DAF922AB3A
:1016260077A878BB01027984BB02027985BB0302E5
:101636007986BB04027992BB05027987BB060279DB
:10164600A3BB0702799CBB08027988BB090279898A
:10165600E8F7227C0512059DDCFB22C2AF1205AD20
:101666001205B41205BB1205C212058E1205AD1283
:1016760005B41205BB1205C212058E1205AD120580
:10168600B41205BB1205C2D2AF22C2AF1205C212F6
:1016960005BB1205B41205AD12058E1205C2120560
:1016A600BB1205B41205AD12058E1205C21205BB9A
:1016B6001205B41205ADD2AF22AE77AF78C2AF1223
:1016C60005AD1205AD1205AD12058EDEF21205C28C
:1016D60012058EDFF8D2AF22D161D159D159757773
:1016E60001757801757900D1BF7C05AD5F12059D46
:1016F600C3ED955F70F5C3E55F9401400AC3E55FEE
:1017060094FF403202171AD125B182D161C2AF755A
:10171600EF12D159DCD50579C3E5799403500280DF
:10172600C6D1590578E5771490009F93F808C3E56C
:101736007898500280AED159D1590577C3E5779490
:101746000A5002809C120EB3B182C2AF75EF12D15D
:011756005939
:0319FD00021002D3
:101A00000E0414FFFFFFFF03040A0301015AA5019E
:101A1000FFFFFFFFFF03FFFFFF25D0FAFA04FF01DE
:081A2000007AFF01010003FF41
:101A400023526F746F724765656B73323041232088
:101A500023424C48454C4923463333302320202031
:101A60002020202020202020202020202020202076
:101C0000C2AFC2D353D9BF7581C043B20343FF8073
:101C1000752438752503B1C975EF0275E24043F1AB
:101C20002053A4DF75D400D2857DFA780379E67C51
:101C300010752200752300901DD67B0675249875BB
:101C400025013085028142208508D8FBD9F9DCF7CF
:101C500081B4308508D8FBD9F9DCF781B4B189E4C7
:101C600093A3C39A6004DDC381B4DBDBB17B600264
:101C7000812B7B08E493FAA3B15CDBF87A30B15C8A
:101C8000752200752300B17BEAFCEBFDC3ED94FEE9
:101C9000400EB17B8A278B28ED30E0048A828B834B
:101CA000B17B7AC270D8C3ED94FE601350CEBD00F4
:101CB00025EC60097520007521FF0200008100A855
:101CC00027A9280809D804D90281D3B17FEA89AAB3
:101CD000F281C50D81A0C3ED94035049EDA2E092BD
:101CE000007AC5C3E5829400E583941C50902000DF
:101CF00010438F02438F0175B7A575B7F1F030001F
:101D00001FA827A9280809438F01538FFDD804D99C
:101D100002A12089AAE275B7A575B7F1F0A3A10DBC
:101D2000538FFC817C7AC1BD030CE493A3FAB140CC
:101D3000DCF8B138817C817EAA22AB23B15CEBFA5E
:101D4000EA6222752608C3E52313F523E52213F57D
:101D50002250066323A0632201D526EAB1C9B1C986
:101D600075260AEAF4200102D285300102C285B14B
:101D7000C9C3134002C201D526EB22B17FEAFB2082
:101D80008502A17F308502A184752608AE24AF2587
:101D9000C3EF13FFEE13FEB1CDB1C9C3EA13308513
:101DA000024480FA30E703632201C3E52313F523DD
:101DB000E52213F52250066323A0632201D526D91C
:101DC000E52265236523F52222AE24AF250E0FDE22
:101DD000FEDFFCD20122424C48656C693437316326
:041DE000F3300601D5
:00000001FF
